:1000000042C0B5C15BC05AC059C058C057C056C0E5
:1000100055C054C053C052C051C050C04FC04EC054
:100020004DC04CC04BC04AC049C048C047C046C084
:1000300045C044C009021200010100A019090400D2
:1000400000000000000012011001FF000008C016AF
:10005000DC050401010200010E03550053004200BB
:100060006100730070001C037700770077002E009A
:10007000660069007300630068006C002E00640075
:1000800065000403090411241FBECFEFD4E0DEBFD6
:10009000CDBF11E0A0E0B1E0E8EBF5E102C00590D2
:1000A0000D92A630B107D9F721E0A6E0B1E001C07A
:1000B0001D92A035B207E1F76EDA7CCAA1CFCF93CB
:1000C000DF9360912E01635067FDB7C080912B01D3
:1000D000CCE0D0E0C81BD109CE5CDE4F80912A0174
:1000E0008D3209F096C0683009F0A5C083EC80938A
:1000F0001E018AE5809302011092060188818076B4
:1001000041F0CE01FBD48F3F2FEF920709F46DC071
:1001100075C09A81109227018981811107C01092C0
:10012000280127E231E082E090E05AC0853019F4DE
:1001300090932F0142C08630D1F58B81813019F424
:1001400086E490E004C0823049F484E390E0909328
:100150002D0180932C0182E190E025C0833009F5C8
:10016000911109C082E890E090932D0180932C01B9
:1001700084E090E018C0913049F486E690E09093D6
:100180002D0180932C018CE190E00DC0923049F458
:1001900088E590E090932D0180932C018EE090E013
:1001A00002C080E090E020E42093060127C0883060
:1001B00099F0893039F49093310127E231E080E001
:1001C00090E00EC031E020E08A3009F030E0832F6B
:1001D000922F27E231E004C021E331E081E090E09A
:1001E00030932D0120932C0109C0288127FF02C0E4
:1001F0008E819F8120E82093060106C02E813F81D9
:100200002817390708F4C901909301018093000170
:1002100012C08091060187FF0EC0CE0177D78F3FB5
:1002200021F48EE18093020106C0882321F0109210
:1002300001011092000110922E018091020184FFB1
:1002400062C080910001909101018F3F2FEF9207D2
:1002500009F459C0BC018930910510F068E070E0E4
:10026000861B970B909301018093000190911E01D2
:1002700088E8892780931E01C62F662309F44EC0A3
:100280002091060127FF07C08FE191E041D6C82FDA
:10029000893080F521C080912C0190912D0126FF9D
:1002A00009C0AFE1B1E0FC0124912D93319661507A
:1002B000D9F707C0DC01EFE1F1E02D912193615006
:1002C000E1F72FEF2C0F30E02F5F3F4F820F931F8E
:1002D00090932D0180932C016C2F8FE191E043D0FE
:1002E000CC5FCC3071F08FEF9FEF90930101809342
:1002F000000107C08FEF9FEF9093010180930001F1
:10030000CEE1C093020184E196B3937069F4815009
:10031000D9F710922F011092290106C060E08FE1F9
:1003200091E021D0C4E0DFCFDF91CF91089585B770
:10033000836085BF8BB780648BBF0895A82FB92FCA
:1003400080E090E041E050EA609530E009C02D91F6
:1003500082279795879510F084279527305EC8F3FC
:100360006F5FA8F30895EADF8D939D930895CF936F
:10037000CFB7CF93C395189BE9F7189B09C0189B7B
:1003800007C0189B05C0189B03C0189B01C0A1C0E3
:10039000DF93C0912B01DD27CE5CDE4F189B02C09E
:1003A000DF91EBCF2F930F931F9303B12FEF00FB40
:1003B00020F94F933F9313B14FEF012700FB21F931
:1003C0003BE031C04E7F012F13B1216028C0102FB8
:1003D0004D7F2260000003B129C04B7F2460012FB4
:1003E000000013B12BC013B1477F28602AC04F7E95
:1003F00003B120612CC04F7D13B120622FC04F7B11
:1004000003B1206432C0422703B149934FEF00008B
:10041000102710FB20F913B11370C9F1297F91F255
:10042000012700FB21F903B1237F89F2315058F1F4
:10043000102710FB22F913B1277E79F2012700FB68
:1004400023F92F7C81F203B1102710FB24F92F79B7
:1004500071F200C013B1012700FB25F92F7359F287
:1004600000C003B1102710FB26F9223040F200C073
:1004700013B1012700FB27F9243028F64F772068B5
:1004800013B10000F9CF11E01CBB002717C03B508F
:100490003195C31BD04011E01CBB0881033CE9F03F
:1004A0000B34D9F0209129011981110F1213EDCFCE
:1004B000093641F10D3211F0013E39F70093300158
:1004C0003F914F911F910F912F91DF91CCB3C0FDC0
:1004D00051CFCF91CFBFCF911895209130012223DA
:1004E00079F310912E01112311F5343012F130936C
:1004F0002E0120932A0110912B013BE0311B3093F8
:100500002B0117C000912E0101308CF40AE53091C7
:10051000020134FD10C000930201CEE1D1E00FC012
:100520002795A8F45150A9F4220F0000F9CF4AE50D
:1005300003C042ED01C0432FC4E1D0E032E014B16A
:100540001360289A14B905B120E413E05F930127E2
:1005500056E005B9279520F4515021F4220FF9CF28
:10056000012756E000003B5A05B9D0F2279528F440
:10057000515029F4220F0000F9CF012756E02795AA
:1005800005B920F4515021F4220FF9CF012756E08C
:100590002991332305B921F60C7F10912F01110FFA
:1005A000C651D04005B911F01093290111E01CBBD0
:1005B000016014B11C7F402F4C7F5F9100C000C0D0
:1005C00005B914B945B97CCF8FB9779BFECF8FB1F0
:1005D0000895DC01CB0121E1B695A7959795879504
:1005E0002A95D1F720914C012817D9F080934C011E
:1005F000E0914901F0914A018DE40995E0914901AA
:10060000F0914A0180E00995E0914901F0914A0199
:1006100080914C010995E0914901F0914A0180E0F7
:100620000994089580914B018DB9809148018EB94C
:100630000895882319F0883060F101C08AE024EE23
:1006400032E030934A01209349011092480191E031
:1006500090934D018B3071F028F48830B1F08930DF
:1006600091F00AC08C3021F08D3031F480E50EC05D
:100670009093480181E50AC082E580934B0181E0B7
:1006800080934801089582E501C083E580934B0182
:10069000089521E733E030934A01209349018430E3
:1006A00081F030F4823079F0833079F480E30EC049
:1006B000863061F020F0873041F483E007C08CE0A1
:1006C00005C088E103C080E601C080EC80934D0145
:1006D000089522B790914D0182B7821B8917E0F3EC
:1006E00008951F93CF93DF93182FD8E0C0E017FF32
:1006F00002C0C39A01C0C398110FCC0FB499CF5F49
:10070000C59AE7DFC598E5DFD15089F78C2FDF91D7
:10071000CF911F91089587B38C6287BBC298C5980B
:10072000D8DFC29AD6DFC2988091490190914A01E0
:10073000845E924009F476DF10924C01089587B3ED
:100740008C6287BB8091490190914A01845E9240FE
:1007500009F468DFC298089587B3837D87BB88B3A7
:10076000837D88BB1DB80895CF93DF93C1E2C1504C
:1007700051F1E0914901F0914A018CEA0995E0912B
:100780004901F0914A0183E50995E0914901F09111
:100790004A0180E00995D82FE0914901F0914A0182
:1007A00080E00995D33589F01DB893DFC29A91DFB7
:1007B000C2988FDF8091490190914A01845E9240F6
:1007C000B1F630DFD4CF81E001C080E0DF91CF917E
:1007D0000895CF92DF92EF92FF926B017C01F9DED8
:1007E0008C2D8170880F880F880FE0914901F0915E
:1007F0004A0180620995D701C60129E0B695A795FF
:10080000979587952A95D1F7E0914901F0914A0192
:100810000995D701C601B695A79597958795E0915B
:100820004901F0914A010995E0914901F0914A018D
:1008300080E0FF90EF90DF90CF900994CF92DF920D
:10084000EF92FF92CF93DF936B017C01C42FD22FE5
:10085000C0DE8C2D8170880F880F880FE0914901D0
:10086000F0914A0180640995D701C60129E0B69547
:10087000A795979587952A95D1F7E0914901F09131
:100880004A010995D701C601B695A7959795879511
:10089000E0914901F0914A010995E0914901F091F7
:1008A0004A018C2F0995DD2321F0CF3721F48FE009
:1008B000A6D080E00FC0D2B7CEE1C701B60189DF74
:1008C0008F37B9F782B78D1B8D33B8F3D2B7C150CC
:1008D000A1F781E0DF91CF91FF90EF90DF90CF9073
:1008E0000895CF92DF92EF92FF92CF93DF936B0147
:1008F0007C01C42F6EDEE0914901F0914A018CE445
:100900000995D701C60129E0B695A79597958795D2
:100910002A95D1F7E0914901F0914A010995D70153
:10092000C601B695A79597958795E0914901F091F5
:100930004A010995E0914901F0914A0180E0099549
:10094000CF3F19F48FE05BD010C0D2B7CEE1C70122
:10095000B6013FDF8F3F49F482B78D1B8D33B8F36B
:10096000D2B7C150A1F781E001C080E0DF91CF9103
:10097000FF90EF90DF90CF900895CF93DF93EC013D
:10098000E0914901F0914A0180EA0995E09149011D
:10099000F0914A018D2F0995E0914901F0914A01AA
:1009A0008C2F0995E0914901F0914A0180E0DF9197
:1009B000CF9109941F93CF93DF93D82F192FC62F70
:1009C000E0914901F0914A0180EC0995E0914901DB
:1009D000F0914A01812F0995E0914901F0914A0176
:1009E0008D2F0995E0914901F0914A018C2F0995CD
:1009F0008EE105D080E0DF91CF911F91089590E0C6
:100A0000981739F032B722B7231B2C33E0F39F5FDE
:100A1000F7CF089590E0981739F032B722B7231B2B
:100A20002B3BE0F39F5FF7CF0895259A23982B9AED
:100A300050E217D05A95E9F70895AC0188E605D041
:100A4000842F03D089E601D0852F0FD028E030E035
:100A5000382780FB869506D02A95D1F730FB02D047
:100A600000D0689423982B9A16F02B98239AE09143
:100A70004E01F0914F013197F0F72D9AE3B1E3FB6E
:100A8000E0914E01F0914F013197F0F72D980895C4
:100A900020ECE7DF46F42A95E1F780E02AE1E5DF84
:100AA0002A95E9F7DECF28E030E0DBDF869587F98D
:100AB00038272A95D1F7D5DF27F9322772F3D1DF0E
:100AC000D0CFDB01742FB9DF84E2BFDFE1DF8D938C
:100AD0007A95D1F70895DB01742FAFDF83EFB5DF8F
:100AE0008DE1B3DF84E6B1DF8D91AFDF82E7ADDF6B
:100AF000CFDF8078D9F77A9589F70895CF93DF9380
:100B0000EC018981813061F4329902C085E002C034
:100B1000809114018EDD109213014198FCDDEDC12E
:100B20008B3319F48A8176DFE8C1823351F432992C
:100B300002C085E002C0809114017BDD4198FFDD99
:100B4000DCC1833359F42A989A81909304012E8151
:100B50003F8130930E0120930D01BBC1843361F4BA
:100B60002A988A81809304018E819F8190930E013F
:100B700080930D0182E3ADC1863419F4419830D4DD
:100B8000BCC1893411F431D4B8C18A3411F43ED4D3
:100B9000B4C18C3419F48A8147D462C18B3419F4FE
:100BA0008A8162D45DC1873479F48C81813009F403
:100BB0001CD461E08A8182D48E819F8190930E0142
:100BC00080930D0186E385C1883479F40ED460E00A
:100BD0008A8174D48C81809307018E819F81909348
:100BE0000E0180930D0185E374C18D3579F42A9A45
:100BF0008A81809303018C81809308018E819F817B
:100C000090930E0180930D018AE363C18C3559F4F2
:100C10008A81809303018E819F8190930E0180933E
:100C20000D0189E356C18E3529F48CD4813009F049
:100C3000E9C016C18F3511F492D412C1823011F47B
:100C40008BDD09C18330F9F4E0914901F0914A014B
:100C50008A81099580931601E0914901F0914A013A
:100C60008B81099580931701E0914901F0914A0128
:100C70008C81099580931801E0914901F0914A0116
:100C80008D81099535C18430D1F480911301811192
:100C90000EC08A819B81092E000CAA0BBB0B80938E
:100CA0000F0190931001A0931101B09312018E8156
:100CB0009F8190930E0180930D0182E00AC18730DD
:100CC000D1F48091130181110EC08A819B81092E7C
:100CD000000CAA0BBB0B80930F0190931001A09303
:100CE0001101B09312018E819F8190930E01809328
:100CF0000D0183E0EEC08530D9F436DD8093160116
:100D0000882309F4AFC0C0911401CC2311F0C15065
:100D100001C0C9E0C33008F4A5C08C2F8ADC24DDF3
:100D200080931601C1508111F5CF8C2F82DC9AC0BF
:100D3000863079F58091130181110EC08A819B81E3
:100D4000092E000CAA0BBB0B80930F01909310018E
:100D5000A0931101B09312013C812D81822F8F70DD
:100D600080930A01822F807F40E1849FC00111247B
:100D7000830F911D90930C0180930B0120FD8093B4
:100D800009018E819F8190930E0180930D0181E076
:100D9000A0C0883001F58091130181110EC08A81B5
:100DA0009B81092E000CAA0BBB0B80930F01909323
:100DB0001001A0931101B093120110920C01109236
:100DC0000B0110920A018E819F8190930E018093F6
:100DD0000D0184E07EC0893081F481E080931301AD
:100DE0008A819B81AC81BD8180930F01909310011A
:100DF000A0931101B093120180C08A3031F48A812E
:100E000080931401109216012DC08B3081F48A81D9
:100E10009B8190934F0180934E012A9A229A83E0FE
:100E2000EEDD2A98419880E1EADDFFDD66C08C3076
:100E3000A1F480EC0ADE80E008DE8AE0E0DD2A9A98
:100E400085E0DDDD2A9885E0DADD84B1837D84B933
:100E500085B1837D85B9419A50C08D3031F418DE5B
:100E60008093160181E090E04AC08E3019F48A81A7
:100E7000ECDD43C08F30B1F48A819B81092E000CD8
:100E8000AA0BBB0B80930F0190931001A09311014B
:100E9000B09312018E819F8190930E0180930D017A
:100EA00085E017C08031D1F48A819B81092E000C26
:100EB000AA0BBB0B80930F0190931001A09311011B
:100EC000B09312018E819F8190930E0180930D014A
:100ED00086E0809315018FEF9FEF11C08F3769F483
:100EE00081E0809316019AE1909317011092180106
:100EF0008093190184E090E002C080E090E026E158
:100F000031E030932D0120932C01DF91CF91089592
:100F1000EF92FF920F931F93CF93C62F209115014D
:100F20003EEF320F323008F494C0253009F496C0F9
:100F3000233339F0293309F460C0263309F0DDC0CA
:100F400031C020910D0130910E01462F50E0241741
:100F5000350708F4C22FF82E8C01802F8F198C17BB
:100F600098F4E0914901F0914A0180E00995F80177
:100F700081938F0180910D0190910E0101979093C3
:100F80000E0180930D01E9CF80910D0190910E012A
:100F9000892B09F0B4C080910401882309F4AAC008
:100FA0002A9AA8C020910D0130910E01462F50E0E1
:100FB0002417350708F4C22FF82E8C01802F8F19C3
:100FC0008C1708F09CC080910D0190910E01019743
:100FD00090930E0180930D01892B41F481E044D25E
:100FE000F801808313D21092150104C080E03CD236
:100FF000F80180830F5F1F4FE1CF20910D013091E9
:101000000E01462F50E02417350708F4C22FF82EA2
:101010008C01802F8F198C1770F480D2F801819386
:101020008F0180910D0190910E01019790930E0117
:1010300080930D01EECF80910D0190910E01892BCF
:1010400009F05DC080910301882309F453C077D271
:1010500051C08C017C01E60EF11C40C0462FBC0142
:1010600080910F01909110012CDD80910F019091E2
:101070001001A0911101B09112018C0F911DA11DC1
:10108000B11D80930F0190931001A0931101B093B3
:10109000120135C080911501823021F560910F0158
:1010A00070911001809111019091120192DBF80171
:1010B000808380910F0190911001A0911101B09156
:1010C00012010196A11DB11D80930F019093100193
:1010D000A0931101B09312010F5F1F4F0E151F0552
:1010E000C9F606C080910F019091100146DCDFCF58
:1010F000C83028F41092150102C08FEF01C08C2F68
:10110000CF911F910F91FF90EF900895EF92FF9272
:101110000F931F93CF93C62F20911501213031F4E7
:101120008C017C01EC0EF11CC0E00BC12430C1F33A
:10113000263009F4A6C02233B1F12A3309F462C083
:10114000253309F044C120910D0130910E01462F45
:1011500050E02417350708F4C22FF82E8C01802F99
:101160008F198C1770F4D8018D918D015DD180910C
:101170000D0190910E01019790930E0180930D0146
:10118000EECF80910D0190910E01892B11F080E03E
:1011900021C180910701813011F438D101C025D1DE
:1011A0001092150116C120910D0130910E01462FAC
:1011B00050E02417350708F4C22FF82E8C01802F39
:1011C0008F198C1790F4E0914901F0914A01D801F0
:1011D0008D918D01099580910D0190910E010197DE
:1011E00090930E0180930D01EACF80910D019091B3
:1011F0000E01892B61F680910401882309F4E9C06E
:101200002A9AE7C020910D0130910E01462F50E03F
:101210002417350708F4C22FF82E8C01802F8F1960
:101220008C1708F560910801662389F0683030F466
:10123000F801808149D11092080109C068E0D80105
:101240008C9142D18091080188508093080180914F
:101250000D0190910E01019790930E0180930D0165
:101260000F5F1F4FDBCF80910D0190910E01892BF5
:1012700009F08DCF80910301882309F491CF5FD1CC
:101280008FCF462FBC0180910F019091100123DC7C
:1012900080910F0190911001A0911101B091120164
:1012A0008C0F911DA11DB11D80930F019093100112
:1012B000A0931101B093120180910D0190910E0144
:1012C0008C1B910990930E0180930D01892B09F4D9
:1012D00067CF5DCF80911501813009F051C0209119
:1012E0000B0130910C0160910F0170911001809100
:1012F000110190911201232B41F521E0F801408169
:101300009DDA80910D0190910E01019790930E014D
:1013100080930D01892BE1F180910F0190911001D3
:10132000A0911101B09112010196A11DB11D8093F0
:101330000F0190931001A0931101B09312010F5F60
:101340001F4F0E151F0531F640C020E0D8014C910B
:1013500075DA809109018150809309018111D1CF03
:1013600060910F0170911001809111019091120113
:10137000F8014081B6DA80910B0180930901C1CF59
:10138000D8016C9180910F019091100113DBB9CFBE
:101390001092150180910A0181FF15C08091090109
:1013A00090E020910B0130910C018217930759F0C6
:1013B00060910F01709110018091110190911201C3
:1013C000F80140818EDAC1E0A7CF8C2F03C08FEFE8
:1013D00001C081E0CF911F910F91FF90EF90089590
:1013E000C498C398BC98BB980895BB9A84E18A9529
:1013F000F1F7BC9884E18A95F1F7BB9884E18A956E
:10140000F1F7BC9A84E18A95F1F70895BB9ABC9AEA
:1014100084E18A95F1F7BB9884E18A95F1F7BC984D
:1014200084E18A95F1F7089598E0BB9A87FF02C09E
:10143000BC9801C0BC9A24E12A95F1F7BB9824E13D
:101440002A95F1F7880F915081F7BB9ABC9884E1F7
:101450008A95F1F7BB9824E12A95F1F786B3829536
:10146000817091E089270895282FBB9ABC9834E1B8
:101470003A95F1F7BB9884E18A95F1F796B394FB1E
:10148000882780F997E0BB9A34E13A95F1F7BB9849
:1014900034E13A95F1F7880FB4998160915099F74A
:1014A000BB9A211102C0BC9A01C0BC9894E19A95E4
:1014B000F1F7BB9834E13A95F1F70895613011F4F2
:1014C000816001C08E7FB0CFEF92FF920F931F9388
:1014D000CF93DF9307E010E0061B1109C7E0D0E0CF
:1014E000E82EF12CC017D10791F0C7010C2E02C0D5
:1014F000959587950A94E2F780FF02C0C39A01C0D0
:10150000C398C59AE6D8C598E4D82197EBCFDF9168
:10151000CF911F910F91FF90EF900895CF93DF939C
:10152000D8E0C0E0CC0FC59AD4D8C598D2D8B49929
:10153000CF5FD150B9F78C2FDF91CF910895C2982A
:10154000C598C7C8C29A88E28A95F1F7C2D8B49BF9
:1015500003C0C29880E00895C29881E00895CF93B7
:10156000C29A88E28A95F1F7B4D868E080ECACDFE3
:10157000C0E0C59AAED8B49904C0CA5FC598A9D8CE
:1015800006C0C598A6D8CF5FC83099F7CFEFC298EC
:101590008C2FCF9108951BB815B81AB88FEF84B966
:1015A00014B883E087B99EEF98B985BDC0D678940A
:0815B00086D5FECFF894FFCFB1
:0615B800FFFF5A010100D3
:00000001FF
